:030000000219FDE5
:03000B000200AA46
:03002B0002015D72
:03005B000202FAA4
:030073000202E79F
:1000800002030406080C10182030406080040608A3
:100090000C10182030406080A0C00003070F1F0D17
:1000A0000D04050D050305030302C2AFC0D0C0E077
:1000B000206214E5256009E473E525F4F58AD2622F
:1000C000D0E0D0D0D2AF3285268AC262E526F46075
:1000D0003030682620720DD0E0D0D0C290C291C2DC
:1000E00092D2AF32C290C291C292206F0D20660AA6
:1000F0007401D5E0FDE57BF45290D0E0D0D0D2AFD2
:1001000032758A00C28DD26201FA01B930680520C9
:100110006602D29001B9306805206602D29101B919
:10012000306805206602D29201B9D29330680A2065
:1001300066077405D5E0FDD29001B9D29430680A03
:100140002066077405D5E0FDD29101B9D2953068DB
:100150000A2066077405D5E0FDD29201B9C2AFC28C
:10016000AD53E6EFC0D0C0E0D2D3D2AFC2CEE52AC5
:100170006007207449152A21BE7800790020742E6A
:10018000E580307E01F430E70278FF53DACF207E3D
:100190000343DA20307E0343DA10C2D8C271E5800F
:1001A000307E01F430E70279FFC3E89970CB30610B
:1001B00003752A18207403752A18885CD27020747D
:1001C0000DE52B6004152B21CE43DA01C2D8207037
:1001D00002413DA85C206102C2702074367982B76A
:1001E0000431C3E894F0400374F0F8E8C4540F28D5
:1001F000F87984B703024113C313C313872120087E
:1002000002C313200A06C3C898F8411328F8500304
:1002100074FFF88822E52D54066022206B1FE53616
:10022000C333C333F8E564C313C313F9C395224042
:10023000028922E82522F52250037522FF7882B632
:100240000459852224A824C3E52495614002A861AD
:10025000C3E895634002A8638825E5667002418E75
:10026000C3E8AA669A5003E8FAE4F9EAC333FBE567
:1002700068F45B29400D2567F8E567600215674063
:100280000B418E0AC3E5679A5002056778FF8826FE
:10029000C26FC3E52694F84002D26FC3E5259440AF
:1002A0004002D26420CF0AD0E0D0D043E610D2ADD5
:1002B00032C2CF053A7801E52A6005307402152A6A
:1002C000C3E55C94014005755F0041DD7560007514
:1002D0006900E55F2401F55F5003755FFFD0E0D052
:1002E000D043E610D2AD32C2AF53E67F7592FA75B5
:1002F00093FFC260759104D2AF32C2AF53E6EFC232
:10030000ADC0D0C0E0C0F0D2D3D2AFA8FBA9FCC230
:10031000D8307102616153DACF207E0343DA1030A6
:100320007E0343DA20D271E580307E01F420E702BB
:10033000613888278928A18E53DACF207E0343DADB
:1003400020307E0343DA10C2D8C271307402A17A21
:100350007800E580307E01F430E702A17A885CA164
:100360006253DACF207E0343DA20307E0343DA1073
:10037000C271206102813A53DACF207E0343DA1042
:10038000307E0343DA20C2D8D27188578958C3E837
:100390009555F8E99556F97B007E087A00C3E894F4
:1003A0008CE994005005755B00812C882178A2E6C9
:1003B000A8216055C3E894C8E994005008E4D2E449
:1003C000FB7A0A8107C3E89468E994015008E4D2F3
:1003D000E3FB7A0F8107C3E894D0E994025008E464
:1003E000D2E2FB7A1E8107C3E894A0E99405500885
:1003F000E4D2E1FB7A3C8107C3E89498E994085081
:1004000008E4D2E0FB7A787E00C3E89559FCE995D0
:100410005AFD30E70AECF42401FCEDF43400FD75DC
:100420005B00C3EC9AED9E5003755B018859895AB5
:100430008557558558567802A162C3E89527F8E993
:100440009528F9307C02A146307B02A146307A0221
:10045000A13F207502815DE9FDE8FC817CE9C313C1
:10046000F9E813F8307902A13FE9C313F9E813F86A
:0F047000307802A13FE9C313FDE813FC20612C93
:10047F00C3EC941CED940240028193ED701EC3EC0B
:10048F0094C850180529E52970021529C3E5299448
:10049F000A5002A17A755C00D270A17AE529600238
:1004AF0015297888E6F97400207F087896B9030239
:1004BF00789EE624FAFEE43400FFC3EC9EFCED9F29
:1004CF00FD9208B90310A2085007207609D2768151
:1004DF00E5307602C276A2085016B9030DECF4246B
:1004EF0001FCEDF43400FD0204FF78007900A14611
:1004FF00B90315EC33FCED33FDC3EC940AFCED941A
:10050F0000FD50047C007D00C3EC94FFED9400408F
:10051F000678FF7900A146EC8572F0A4C5F0A2F72A
:10052F0033F87900400302056278FF790002056213
:10053F00E9C313F9E813F8307C0EE9600278FFC3C2
:10054F00E81338F8E43400F9C3E894FFE994004065
:10055F000278FF885CD270206102A17A741FF45573
:10056F002F4BF52FC274EB7002D274752A183074AA
:10057F0003752A0A306102A18E20740353DAFE201C
:10058F007403752B06D0F0D0E0D0D0D2AD43E61077
:10059F003279010205BE79030205BE790A0205BE52
:1005AF00791E0205BE79640205BE79C80205BE78C0
:1005BF0017E4D5E0FDD8FAD9F6227A147B78020534
:1005CF00E57A107B8C0205E57A0D7BB40205E57A9E
:1005DF000B7BC80205E57902E4D294D5E0FDD291F8
:1005EF00D5E0FDC291D5E0FDC294D5E0FDE920E054
:1005FF0002D29030E002D292E573D5E0FDE920E01F
:10060F0002C29030E002C2927496D5E0FDD9C9EAD9
:10061F00F8D5E0FDD8FBDBBED29422C37C007D0071
:10062F0075F00005F0EA33FAEB33FB50F6EB13FBF2
:10063F00EA13FAC3E9FFE8FEE89AF8E99BF95004D8
:10064F00EFF9EEF8B3EC33FCED33FDD5F0DFEDF958
:10065F00ECF822E889F08A20D2D4F8A9F07B003098
:10066F00F70B7BFFF42401F8E9F43400F9E8852057
:10067F00F0A4ADF0F8E98520F0A4AFF0FEED2EF96F
:10068F0074003FFA7C04C3EA13FAE913F9E813F88C
:10069F00DCF48BF030F70AE8F42401F8E9F43400C5
:1006AF00F9E889F0C2D4F8A9F0227882B6040302DF
:1006BF000714C3E55C940140030206DE852224E49F
:1006CF00F544F545F546F547F548C26E020714782F
:1006DF0082E6FCD26EE522F523783879C7AA40ABC3
:1006EF0041C3EB13FBEA13FAEC146013C3EB13FBD8
:1006FF00EA13FAEC14146007C3EB13FBEA13FAD1F5
:10070F002A8844894522C3E5449523F8E54594009A
:10071F00F9500CC3E89480E994FF4016020745C3D3
:10072F00E8947FE994005003020745787F7900022F
:10073F000745788079FF8849894A22E5492546F897
:10074F00E54A3547F9854A20E4300701F43548FA80
:10075F0030E709C3EA94F04015020783C3EA940F08
:10076F00500302078378FF79FF7A0F02078378001F
:10077F0079007AF0C3E5249561500AC3740195247A
:10078F00500B0207A1E54A20E70E0207A1E54A3008
:10079F00E706884689478A482278A5E6FAC3E549DD
:1007AF0033F8E54A33F9D162E930E70BC3E89480B7
:1007BF00E994FF4013E1DBC3E8947FE99400500212
:1007CF00E1DB787F7900E1DB788079FFE820E715BE
:1007DF00C3E52398F84009C3E894014003020802D7
:1007EF007801020802E8F424012523F840030208E7
:1007FF000278FF884B2278A6E6FAA847A948120686
:10080F0062E930E70CC3E89401E994FF401602084F
:10081F0037C3E894FFE99400500302083778FF7953
:10082F0000020837780179FFE920E715C3E54B98F7
:10083F00F84009C3E89401400302085E78010208FA
:10084F005EE8F42401254BF8400302085E78FF8828
:10085F00242278FFC26420693D206A12D264C3E566
:0E086F0041940A4009C3E52594405002C2643A
:10087D0079A1E76023E541601F74FF8541F0848510
:10088D0039F0306A0375F005A4F8C5F0600278FF01
:10089D00C3E895645002A864886322C3E540944080
:1008AD00E5419401E56350031401B9046002F56359
:1008BD00220208C12275E890227883E6FFE5E82040
:1008CD00ECF7A8BDA9BE0570C3E57094084052753C
:1008DD007000E9FA79A0E76044EA7007E571601BE2
:1008ED000208FCC3E895716010E5715006600C14A8
:1008FD000209080460F9020908E571F571C394F65F
:10090D00401B7561C0C394064013756180C3940686
:10091D00400B756140C39406400375610075BB06BD
:10092D0022E5612410500274FFF5617982B704024B
:10093D002155C3A861E524985002A824C3E8956306
:10094D004002A86388258826E570B4070375BB109F
:10095D0022743279A787F0A4C5F0A2F733F8C3E863
:10096D0095614002A861882288248825882688649C
:10097D00227540007541F022C2AF75C820A8CCA9E0
:10098D00CDAA3A30CF010A75C824D2AFAB3BAC3CEF
:10099D00883B893CC3E89BF8E99C206908F93067DE
:1009AD0002419121EEAD3D8A3DF9EA9DFA60047850
:1009BD00FF79FFAE3EAF3F8B3E8C3FA83BA93CC3BA
:1009CD00E89EF8E99FF9C3E54113FBE54013FAE80A
:1009DD002AF540E93BF54150067540FF7541FF4151
:1009ED0038AA40AB41AC40AD417E047F02C3EB94CD
:1009FD000440021E1FC3EB940840021E1FC3ED13DB
:100A0D00FDEC13FCDEF7C3EA9CFAEB9DFBEF6009EE
:100A1D00C3E913F9E813F8DFF7EA28FAEB39FB8A93
:100A2D00408B4150067BFF8B408B41C3EB940250B2
:100A3D0002D2673069047F0341637892E6FFC3E514
:100A4D0037948240110FC3E53794A040010FC3EFD7
:100A5D00940640027F057E02E541C4540FF9E5413D
:100A6D00C454F0F8E540C4540F28F8C3E89EFAE9E1
:100A7D009400FB4009C3EA9402EB940050047A02FF
:100A8D00E4FB41DDAA40AB41EBC4FEEAC4540F4E7A
:100A9D00FCC3EA9CFAEB9400FBC3E813C313F8EA1A
:100AAD0028FAEB3400FB8A408B41C3EB94024002E1
:100ABD00C2677802EBC4FE7B00EAC4540F4EFAC342
:100ACD00EA98FA4005C3940250027A027892E6FF42
:100ADD0030600241DD855192855293D26043E680AC
:100AED00C3E49AF8E49BF93067026169E8FAE9FB1F
:100AFD00D3E913FDE813FC88518952C3EF940360C9
:100B0D0038EF20E00DE82CF8E93DF9ECFAEDFB02A9
:100B1D000B32E828F8E939F9C3E82402F8E9340082
:100B2D00F97AFE7BFFC3EF9403400E8A538B5488F2
:100B3D004D894E8C4F8D50619D885389548A4D8BB4
:100B4D004E8C4F8D503069127553F07554FF754FA3
:100B5D00F07550FF7551F07552FF619DE8FAD3E8BD
:100B6D0013FC8851C3EF94036020EF20E007E82CBD
:100B7D00F8ECFA6189E8282402F87AFEC3EF9403B1
:100B8D0040088A53884D8C4F619D88538A4D8C4FF8
:100B9D00E568C3335002646BF56830600261A77578
:100BAD003402D26043E680E52D54066034A840A996
:100BBD0041C3E913F9E813F8C3E913F9E813F83061
:100BCD006904E92440F9C2AF53E67F759100C3E48F
:100BDD0098F594E499F595759104D26043E680D229
:100BED00AF22D265754300752000306C037520402F
:100BFD00020C0ED265754300752040306C037520D4
:100C0D000078017901206720E52D54066002C26548
:100C1D007914E541C313700104F8C39414400278AC
:100C2D0014306904781B791B206010E543600C308B
:100C3D006903D53404D26D81B171AF0543E59BF4E1
:100C4D005440B52002819B30690908C3E8994001E1
:100C5D0018813520650A08C3E8994002810E813557
:0D0C6D00C265C2AF53E67F7591003067127B
:100C7A007594007595FE759104D26043E680D2AFF3
:100C8A00810EAE40AF41C3E49EF594E49FF5958191
:100C9A0080C3E53394015002810E306502810ED87B
:100CAA000281AF8135C26DC2AF53E67F759100856F
:100CBA005394855495759104854D92854E93D260CF
:100CCA0043E680D2AFE52D54066008206A02053358
:100CDA00020CED306D0D206C0A2065071581158117
:100CEA000215752278003064053065027801E5370F
:100CFA0075F007A4F9E5F028F5F0E9A2F013A2F1DE
:100D0A0013A2F213F537C394785003753778C3E505
:100D1A003795384008D266C290C291C292306002BA
:100D2A00A127854F92855093D26043E68022207D89
:100D3A0016C2AF754202D294C293306202D292D2E4
:100D4A00AF759F11020F27C2AF754202D294C295A6
:100D5A00306202D290D2AF759F11020F27307243D0
:100D6A00207D20C2AF75420390013B757B10C29271
:100D7A00D295306204D291A185C294D2AF759F01F7
:100D8A00020F27C2AF75420390013B757B10C290D8
:100D9A00D293306204D291A1A5C294D2AF759F2199
:100DAA00020F27207D17C2AF754203900116C29227
:100DBA00306202D291D2AF759F01020F27C2AF757E
:100DCA004203900116C290306202D291D2AF759F4F
:100DDA0021020F27207D16C2AF754204D293C29515
:100DEA00306202D291D2AF759F21020F27C2AF752E
:100DFA004204D295C293306202D291D2AF759F015A
:100E0A00020F27307243207D20C2AF754205900140
:100E1A002A757B08C291D294306204D290C12BC247
:100E2A0093D2AF759F11020F27C2AF754205900189
:100E3A004C757B20C291D294306204D292C14BC2CB
:100E4A0095D2AF759F11020F27207D17C2AF754249
:100E5A000590010CC291306202D290D2AF759F11F7
:100E6A00020F27C2AF754205900120C2913062EB92
:100E7A00D292D2AF759F11020F27207D16C2AF758D
:100E8A004206D295C294306202D290D2AF759F01C7
:100E9A00020F27C2AF754206D293C294306202D2C1
:100EAA0092D2AF759F21020F27307243207D20C254
:100EBA00AF75420190014C757B20C290D29330628B
:100ECA0004D292C1D1C295D2AF759F21020F27C217
:100EDA00AF75420190012A757B08C292D2953062A1
:100EEA0004D290C1F1C293D2AF759F01020F27209D
:100EFA007D17C2AF754201900120C290306202D2C2
:100F0A0092D2AF759F21020F27C2AF75420190019D
:100F1A000CC292306202D290D2AF759F01C2662291
:100F2A0090010A757B00C290C291C292D293D29468
:100F3A00D295C26222788076090876090876040872
:100F4A0076FF0876030876FF08760B08760308769C
:100F5A0001087601788C76010876FF0876FF087614
:100F6A00FF0876FF0876FF0876030876FF0876FF03
:100F7A000876FF0876250876D0087628087650087D
:100F8A0076040876FF08760208760008767A0876EC
:100F9A00FF087601087601087600087603087600CD
:100FAA00227887E6FFC272BF0302D2727888E6C34C
:100FBA0094036008C27DE630E102D27DC27E788960
:100FCA00E630E102D27EC3EF94026008758E01D248
:100FDA0073020FE3758E00C273227880E6149000C4
:100FEA00809378A5F67881E6149000809378A6F627
:100FFA007886E61490008D9378A7F67886E6F53918
:10100A00C394025003753902789CE67538FFB4021E
:10101A00037538A0B4030375388278A3E6149000E8
:10102A009A93F566120F2A22227896E6FA7897E6BC
:10103A00FB7888E6B40305C3EB940EFB307F047A91
:10104A00007BFFC3EB9AFCC3948250027C827572C8
:10105A00000572EC8572F0A4C3E5F0947D40F2229B
:0D106A00D27F11331205AF7A007B007C109D
:101077001205A5E55C2AFA74003BFBDCF37C04C38C
:10108700EB13FBEA13FADCF7FEC27F113322E5EF1D
:1010970020E6037520000520903FFFE52014600639
:1010A700901DFF1460009304600375EF1053D9BFC0
:1010B7007581C043FF801205A075EF0043B203E5B9
:1010C700B3240220E70DF521E5E320E0068521B3EF
:1010D70043E301120F2A7580FF75A40075F190751F
:1010E700D47F75903875A53F75F23F75D50075A605
:1010F7000175E241120F2AE4F8F6D8FD756801126E
:101107000F3F1215C678988673753001C2AF120566
:10111700B91205C91205AF1205D01205AF1205D7CE
:101127001205AFC2AF78FA79FA308707D9FBD8F73B
:10113700021C00120FAB120FE4113211337898869C
:1011470073120F2A75881075890275C82475910462
:1011570075D84075A82275B80275E690759B80759D
:101167009D0075D10775BC5875BB0675BA1175E832
:10117700801205A0D2AF1208BE75360053DACF2011
:101187007E0343DA20307E0343DA1043DA01C2D804
:10119700C2711205B9D2617B037A0CE55B70077ADD
:1011A7000CDB0302112A1205AF20700302112AC2B9
:1011B70070E55CC3940240E1E52F541F855E5DF541
:1011C7005EB55DD5DAD5C26153DACF207E0343DA47
:1011D70020307E0343DA10C2D8C27178A2E67008C5
:1011E700D274E52F54E0F52FC2757529001205B4A6
:1011F700307409C3E529940A4002D2751205A5780F
:10120700023074027800C3E55C9840F0C2AF120563
:10121700C91205C91205C9D2AF1205B9754C0078B4
:1012270088E6B4030261021205A5788CE6C394012F
:101237005003021302E530C3940150030213022046
:101247007435C3E55C94FF5003021302C2AF120565
:10125700DED2AF1205B4C3E55C940150EFC2AF1202
:1012670005C91205AA1205C9D2AF1205B4C3E55CB8
:1012770094FF40E902176E7F02D27F11331205B443
:10128700C2AFC27F1133AE5CC3E55C947FD2AF407F
:10129700741205A0C2AF1205DED2AFDFDC116AC33C
:1012A700EE7897F61205B91216081216F17F0AD2D0
:1012B7007F11331205B4C2AFC27F1133AE5CC3E5F1
:1012C7005C947FD2AF50E61205A0C2AF1205C912D7
:1012D70005AA1205C9D2AFDFD6116AEE24037896A4
:1012E700F61205B91216081217201205B41133C3E6
:1012F700E55C94FF5002414602176EC3E55C954CCE
:101307004003855C4C1205B478017988E7B4030281
:101317007805C3E55C9840024126C2AF1205DE128C
:1013270005DE1205DED2AF1205B9753000E4F531DE
:10133700F5320531E531F4703F0532789AE67819D0
:10134700146012783214600D787D14600878FA14EE
:101357006003753200C3E53298401D120F2A12054B
:10136700A0153275310078998673C2AF1205DED2A7
:10137700AF789886731205B41205AAE52A7005306E
:101387007402212A78012074027806C3E55C98402C
:10139700A17888E6C3940360031205B4E52A7003B5
:1013A70002112AC2AF120F2AE4F522F523F524F51C
:1013B70025F526F567D2AF7885E6C333F565E4F5FD
:1013C70044F545F546F547F548F570F52CF52DF547
:1013D7003775700875BB101205A01208C2E5E82022
:1013E700ECFBA8BDA9BEE97001F888711208C675A3
:1013F700700875BB10120FABC2AF7561FF12095EA3
:10140700852261852262852263D2AF752201752408
:1014170001752501752601856069756A017888E679
:10142700B40307C27D307602D27DD268D2697533A4
:1014370000120E84120EB312097E12098512097E5C
:1014470012098512097E120C001206B9120CEE124F
:101457000D38120985120BEF306E0312071520673E
:0D146700031208613067031208A8120CEE92
:10147400120D67120985120C00306E0312074A120E
:101484000CEE120DDE120985120BEF306E031207FB
:10149400A8120CEE120E0D120985120C00306E0308
:1014A400120805120CEE120E841209851208C212DB
:1014B4000BEF120CEE120EB31208C6120985306936
:1014C40032856461856462856069756A0179187A18
:1014D4000CC3E53399400FC269D26A8A35856461C9
:1014E4008564630214F7C3E55C9401400302144D60
:1014F40002157D306A1D206C1AE535147006C26A27
:10150400D26B814DF535C3E55C9401400302144D63
:1015140002157D75360078FA79A4E760027803C372
:10152400E55F985054307404E52A604D7888E6B439
:101534000317207D05207607A14D307602A14D20AA
:101544006C07D26C856461818C78F0306C0585649D
:10155400617820C3E541985002814D306C1BC26C08
:10156400C27D307602D27DD26A753512856461817E
:101574004D0536E55C6002A180753600C2AF120FDE
:101584002A7887E6FE7602120FAB7887EEF6E4F54A
:1015940022F523F524F525F526F565752C00752D22
:1015A40000D2AF1205B4120F2A78A4E66006D290D6
:1015B400D291D292307409C3E53694044002212AB0
:1015C4006134901A0D782012164AE520B4550CA304
:1015D40012164AE520B4AA030215E8120F3F1216A8
:1015E40008021607901A0378807B0A12164AA30889
:1015F400DBF9901A0F788C7B1912164AA308DBF9D1
:10160400901A2822C2AF121689121663901A007417
:101614000E12164FA3740612164FA3741512164F0A
:10162400901A0378807B0A12164EA308DBF9901AED
:101634000F788C7B1912164EA308DBF912169C1234
:10164400167A901A2822E493F622E6438F01538FE8
:10165400FD75EF0275B7A575B7F1F0538FFE224300
:101664008F02438F0175EF0275B7A575B7F1901A14
:101674000DF0538FFC22901A0D7455D14F901A0E11
:1016840074AAD14F227A3079D07820901A40D14A66
:10169400E520F709A3DAF7227A3079D0901A40E7E7
:1016A400D14F09A3DAF922AB74A875BB0102798082
:1016B400BB02027981BB03027982BB04027984BB39
:1016C40005027986BB06027992BB07027987BB08BB
:1016D4000279A3BB0902799CBB0A027988BB0B027D
:1016E4007989E8F7227C051205B9DCFB22C2AF1226
:1016F40005C91205D01205D71205DE1205AA120576
:10170400C91205D01205D71205DE1205AA1205C9A1
:101714001205D01205D71205DED2AF22C2AF1205D0
:10172400DE1205D71205D01205C91205AA1205DE6C
:101734001205D71205D01205C91205AA1205DE1228
:1017440005D71205D01205C9D2AF22AE74AF75C247
:10175400AF1205C91205C91205C91205AADEF21293
:1017640005DE1205AADFF8D2AF22D1F1D1E9D1E921
:10177400757401757501757600F14F7C05AD5C12C9
:1017840005B9C3ED955C70F5C3E55C9401400AC3EB
:10179400E55C94FF40320217AAD1ABD108D1F1C263
:1017A400AF75EF10D1E9DCD50576C3E57694035027
:1017B4000280C6D1E90575E5741490009F93F8087A
:1017C400C3E57598500280AED1E9D1E90574C3E54B
:1017D40074940C5002809C120F3FD108C2AF75EF75
:0317E40010D1E938
:0319FD0002109540
:101A00000E0615090904FF03FF0B03010155AA0186
:101A1000FFFFFFFFFF03FFFFFF25D0285004FF0259
:091A2000007AFF0101000300FF40
:101A40002345415A5933417632232020202020203B
:101A500023424C48454C4923463333302320202031
:101A60002020202020202020202020202020202076
:101C0000C2AFC2D353D9BF7581C043B20343FF8073
:101C1000752438752503B1C975EF0275E24043F1AB
:101C20008053A47F75D4FFD2877DFA780379E67C50
:101C300010752200752300901DD67B0675249875BB
:101C400025013087028142208708D8FBD9F9DCF7CB
:101C500081B4308708D8FBD9F9DCF781B4B189E4C5
:101C600093A3C39A6004DDC381B4DBDBB17B600264
:101C7000812B7B08E493FAA3B15CDBF87A30B15C8A
:101C8000752200752300B17BEAFCEBFDC3ED94FEE9
:101C9000400EB17B8A278B28ED30E0048A828B834B
:101CA000B17B7AC270D8C3ED94FE601350CEBD00F4
:101CB00025EC60097520007521FF0200008100A855
:101CC00027A9280809D804D90281D3B17FEA89AAB3
:101CD000F281C50D81A0C3ED94035049EDA2E092BD
:101CE000007AC5C3E5829400E583941C50902000DF
:101CF00010438F02438F0175B7A575B7F1F030001F
:101D00001FA827A9280809438F01538FFDD804D99C
:101D100002A12089AAE275B7A575B7F1F0A3A10DBC
:101D2000538FFC817C7AC1BD030CE493A3FAB140CC
:101D3000DCF8B138817C817EAA22AB23B15CEBFA5E
:101D4000EA6222752608C3E52313F523E52213F57D
:101D50002250066323A0632201D526EAB1C9B1C986
:101D600075260AEAF4200102D287300102C287B147
:101D7000C9C3134002C201D526EB22B17FEAFB2082
:101D80008702A17F308702A184752608AE24AF2583
:101D9000C3EF13FFEE13FEB1CDB1C9C3EA13308711
:101DA000024480FA30E703632201C3E52313F523DD
:101DB000E52213F52250066323A0632201D526D91C
:101DC000E52265236523F52222AE24AF250E0FDE22
:101DD000FEDFFCD20122424C48656C693437316326
:041DE000F3300601D5
:00000001FF
